:100000008316BF3087008601243098008130990024
:10001000831290309800FF3086005920003086000F
:10002000A60126081A20003E031919284220A60A14
:10003000112819288207533450344534433454343A
:10004000523455344D342034933464348E34713406
:100050008D3448348D34EC348234CC3483347A3467
:1000600081345B34833480348334793481345B3439
:100070008334573400340034003400340034003406
:1000800000340034A5008316981C442883122508E8
:1000900099000800A530A00000000000A00B4E2829
:1000A00008006330A100000000004A20A10B552881
:1000B00008006330A2006230A3000330A4000000F7
:1000C0005120A20B60284A20A30B6328A40B6628AA
:0200D000080026
:00000001FF
